:1074000080E189BD82E189BD09B400FEFDCF089508
:10741000AA2069F08091E9008F931092E900A9D425
:1074200083FF01C028D58F9187708093E90008956C
:107430008EEF0090E10008220092E1000895F20131
:10744000F999FECFF2BDE1BD0895F9DFF89A80B554
:1074500008C0F5DF1FBA80BD0FB6F894FA9AF99A02
:107460000FBE31962F010895E0E0F0E085919491F0
:10747000019608958BEA36D089EE34D010928900B7
:107480008AEF8093880082E080936F0083E080938E
:107490008100EBE6F7E7859130D0E737E1F781E04F
:1074A0008093D7008AE482BF1092D8001092E20045
:1074B0001092DA001092E10080E808D019BCAA24EA
:1074C0001092E0006CD489E05DD481E98093D8000B
:1074D0000895A3E6B1E090E810D08D939A95E1F776
:1074E000089586E008D015C083E005D08F2F05D021
:1074F0008E2F03D080E05E9A72988EBD8DB587FF87
:10750000FDCF8EB5089505D085E0F5DFF6DF80FD6F
:10751000FDCF729A5E9808958FE08221E9F7F9DF36
:10752000E3E6F6E090EB5C98892FE7DF80E1E5DFAA
:107530005C9A8191E2DF83E68E278F77D1F793956E
:10754000983B89F70895E3E6F1E097FC36C094FC98
:107550004DC092FE089596849920D1F3F894C08985
:10756000D78520E030E080E090E4AFEFBFEF1196E8
:1075700089199040E0F72D01BD4F8D0127FD13C003
:10758000E0E0F8E011928EE7819392E4E1179193A5
:107590009AE508F092E4E334C9F781931082BFDFE3
:1075A000FE012196A1DF95DFF90107D520583F4F55
:1075B000040D151D9A9411F724C28301282D6090A3
:1075C0006C0170906B0143D019F48823C1F70895C2
:1075D000380188243CD0C9F580916A01821709F4EA
:1075E000830160906E0170906D01F4CF80E1982E60
:1075F00060906E0170906D012AD059F48823B1F724
:1076000008959FEF95FC03C096FE089591E097FBC7
:10761000890E662477248301222719D0B1F48823A8
:10762000A1F380916A0136F0881650F4821730F089
:10763000213003C0881520F4281710F48301282F67
:1076400060906E0170906D01E8CF3801822EF301D9
:107650004BDF3FDFC3E6D1E0E4E6F7E70990859131
:10766000081621F4EB36D1F70880801052CFC9E01C
:1076700032DFCA95E9F7D0E195FC1EC094FC37C013
:1076800096FE51C0C3E6D2E0E3E6F6E098E088E774
:107690008E0F00840192E817E1F7884F099001925C
:1076A000E817E1F7C858DF4F9A9589F735DFC85FCB
:1076B000D340C33E49F749C0C3E6D6E0EBE5FAE064
:1076C00098E08E2F885702900086E817E1F73896E9
:1076D0000A900292E817E1F73897C857D0409A9578
:1076E00081F71ADFC850DC4FC33E41F72EC0A3EE2E
:1076F000B6E0E3E6F6E09AE0C6E00D9080818025F2
:10770000807F802582958193A336B90709F4B2E082
:10771000E336F90709F4F2E0E336FC0771F7FCDE23
:10772000DA9529F712C0A3EEB9E0E3E6FAE092E0B9
:107730000E90829180258F70802582958083E3361C
:10774000F907B1F7E9DEDA9571F78827089580E83F
:1077500080BF8DEA8093640089E98093650085E0AD
:1077600083BF889541524455424F59D5F08D14A19D
:10777000C881CFD9F1AF000000FFFFCFCFFFFFFFDF
:10778000FFCFCFFFFF0000FE067E7E06FE46565668
:1077900016FE0656461EFE3F61E9E3FFE3EBE3FFFC
:0877A000E3EBE3FFE16B3F00A6
:1077A8001201100102000008412336000100000008
:1077B800000109023E0002010080320904000001B4
:1077C8000202010005240010010424020405240615
:1077D8000001070582030800FF09040100020A00EE
:1077E80000000705040210000107058302100001CC
:1078000011241FBE04B714BE88E1E0E6F0E08083D7
:1078100011928EEF9AE09EBF8DBF22243324210166
:107820003101410151018AC00F928F939F931F92A2
:107830000FB60F9211244F936F938091DA0080FF5F
:1078400037C023C00F920FB68F939F93EF93FF9390
:1078500088278093850080938400E0E5F1E09281A1
:10786000907261F490818917980B908309F45D9A66
:1078700091818917980B918309F4289A239411F424
:107880008315381EFF91EF9154C08091D80080FF7E
:107890000FC08091DA008E7F8093DA008091D9004A
:1078A00080FF04C0ADDD81E0A82E02C019BCAA246F
:1078B0008091E10080FF0BC05FD280FF08C05FD2E3
:1078C0008091D800806202DE19BC85E0A82E8091EC
:1078D000E10084FF1AC050D284FF17C091DD80916F
:1078E000D8008F7DF3DD8FEEA4DD46D28F7E8160E0
:1078F00049D280915301882331F48091E30087FDC0
:1079000002C081E001C084E0A82E8091E10083FFE5
:107910000CC032D283FF09C087EF8BDD82E0A82E36
:107920001092530185DD2BD23AD26F914F910F9077
:107930001F909F918F910FBE0F90189580E88083C4
:107940001082B1E0B5BF82E085BF81EF85B987EED7
:1079500084B984E08DB984E48EB910BA83EF81BB19
:1079600080E68BB980EF8AB980E58CBDBDBDA0E013
:10797000E8EAF7E705900D92A035E1F78C911D92AA
:10798000BB30E1F7893B11F4ADDDE1CE5F9A04C075
:107990007C9B02C069DDA9F56DDD789449D071F05A
:1079A000ABE9B7E0E7E7F7E790E105900D929A952C
:1079B000E1F7A059BF4FE73AB9F7B2DD67D028DD4C
:1079C000809152018078C9F48FB18095807F66994B
:1079D0001C9B8460982E15DE89EB88258093FF0A16
:1079E0008110B1DD882049F492FC09C00B2C97FC72
:1079F000BA9494FCB394B010D1CF3320FAF634DDAE
:107A0000E9F2F89489EB6EDD81E08093E00010925A
:107A10006F0010928100109285001092840085BF43
:107A200015BE2E9A2F9A2D9A5D9A289A0C940000D2
:107A300058DD85EC60DD8B2D55DD662477248824A8
:107A400006CE95D107C046D102C0AA2039F091D107
:107A500082FFFBCF85FFF7CF8091F1000895082EBC
:107A600083E086D185FD07C07BD102C0AA2069F0E2
:107A700080D180FFFBCF0092F10080915201807293
:107A800021F45D9884E680935001089570D182FFBF
:107A900023C180915201807221F4289884E680935A
:107AA0005101CFDF182F853431F422248EE7382E90
:107AB000C6DC8DE0FAC0843521F4C3DFB82EB8DF10
:107AC000F8CF8C34B1F38035A1F3843711F480E022
:107AD000ECC0813429F4B5DF582EB3DF482EE9CF4E
:107AE000833539F4E4E6F7E78591B9DFEB36E1F762
:107AF000DDC0863521F482E3B2DF81E3D6C086376C
:107B000061F481E3669B8E5F1C9B8F5FA8DF8FB162
:107B1000809582958F708F5BC8C08837A9F491DFFC
:107B200080935201289A84FD28985D9A83FD5D9880
:107B30002E9A81FD2E982F9A82FD2F982D9A80FDE6
:107B40002D9887FD8824B5CF8A3649F48FE9D3DC98
:107B5000C3E0D3DC84DFCA95E1F7DBDCA7C0833761
:107B600031F487E87CDF85E97ADF8EE19EC08236DA
:107B700031F489E574DF80E072DF80E896C08234FA
:107B800019F0873609F07DC033245BDFD82F59DF29
:107B9000C82F57DF082F8354843008F085C006347F
:107BA00011F4440C551CF20110926F001736B9F411
:107BB000033489F483E099DCA0DC8EB51EBC4FDF72
:107BC0000DB42197D1F7A5DC08C0063411F48591D6
:107BD00001C03BDC44DF2197C2F72F014AC00334C8
:107BE000A9F4E11104C07DDC88ED7FDC8CDC79DC5C
:107BF00082E07BDC26DF0DB48EBDCA95D9F73196C5
:107C00007DDC81DCDA9569F72F0131C00634F1F4AF
:107C10009F01F437D8F4E4D119C013DF063461F4BE
:107C2000C0FB46F0F43728F4182E81E087BFE895B2
:107C300011243296082E0AC0043439F4DF01B370DF
:107C4000AD59B94F8D93319601C003DC21972AF7C6
:107C5000043431F42F01F370FE2B49F461DC07C0CA
:107C6000063429F42F01F901F43708F4B7D18DE077
:107C7000F6DE063411F45694479482E080936F0048
:107C800015C08237E1E049F08634E0E031F08E340F
:107C9000E3E019F0813531F4E2E0F0E089E087BFFC
:107CA000849103C08B3111F08FE3D9DE83E0BDDB1B
:107CB00057D095FF03C009C0AA2071F05AD080FFA9
:107CC000FBCF4ED002C0AA2039F053D080FFFBCFAB
:107CD00084E0ABDB8BE745C00895E4E5F1E067E0C5
:107CE00090915B0180915C01913231F0913AF1F514
:107CF0008132E1F560D183C0823281F48191805B71
:107D00008191844099F580915D0180FD2FC0F894A8
:107D100081E08093E0001092FF0A72CD803231F54D
:107D20004AD1AA20E9F08530D9F023D083FD18C0CC
:107D300082FFF7CF04C090DE8193615031F09091C3
:107D4000F3008091F200892BB1F7C4DF611549F788
:107D500004C0AA2029F0853019F00BD080FFF9CF9C
:107D60008EE79091E80089238093E800089584E0ED
:107D70005CDB8091E80008958091E2000895FCDFCB
:107D80008E7F80618093E200089582E061EC09D0EB
:107D900083E061E802D084E060E842E103C080E073
:107DA00060E042E042DB81E007D01092ED0060939A
:107DB000EC004093ED0008959091EB00892B8093A7
:107DC000EB00089560E0923029F0913029F4E0E072
:107DD00062E102C0E2E16EE3F1E0089580915B01AF
:107DE00088234CF402C0AA20C1F3C3DF82FFFBCF7B
:107DF00071CFAA2091F3BDDF80FFFBCFB1CF4091BF
:107E00006101509162014617510520F0462F61151E
:107E100009F4A6DF50E022C0AA2061F1853051F1BB
:107E2000A8DF83FD57CFA5DF82FD21C080FF16C0EC
:107E30003091F3002091F20006C081918093F1000F
:107E400041502F5F3F4F411519F028303105A8F3FD
:107E500050E02830310509F451E082DF4115E1F6A8
:107E60005523D1F604C0AA2029F0853019F081DF0E
:107E700082FFF9CF2FCFEBE5F1E0EEDD8193E33622
:107E8000E1F72BDF76DF83FF91C080915B0190915A
:107E90005C01913009F170F09330F1F0953009F404
:107EA00044C0963009F456C0983009F460C0993047
:107EB00059F767C0823841F780915F01B5DA2091A8
:107EC000EB001092E90077D022952695217020933F
:107ED000F1001092F10052C0882311F08230A1F617
:107EE0008F71823089F680915D018823D1F42091D1
:107EF0005F01277049F22093E9008091EB0080FF39
:107F000010C0933011F480E20BC080E155DF81E0B6
:107F1000880F2A95E9F78093EA001092EA0088E03A
:107F20004BDF1092E90047D02AC0882391F41091CA
:107F30005D0110680FB7F8943ED050DF1ADF80FF64
:107F4000FDCF1093E300103883E009F482E0A82EFF
:107F50000FBF2CC08058823048F580915D01909110
:107F60005E0130DF603011F126D049DF1FC080385C
:107F7000E9F421D0809153018093F100F1DE2EDFEE
:107F800015C0882399F490915D01923078F4909314
:107F9000530111D023DF80915301882321F4809174
:107FA000E30091E087FD94E0A92EEFDEE2DE83FF9F
:107FB000089580E201DF87EFD4CEA3E6B1E0F43785
:107FC000B8F40ED090E40D901D9081E087BFE89545
:107FD00032969A95C1F71124E058F04085E001C02F
:107FE00083E001D081E187BFE89507B600FCFDCFB3
:027FF0000895F2
:067FFA003231E0CFFBDC98
:040000030000740085
:00000001FF
